:06000000008076022BD8FF
:03000B0002245E6E
:030013000223388D
:03001B0002255B60
:03002300022B812C
:10002B0032534D50544520496E7465726661636559
:10003B002020202863292031393935202020416C9C
:10004B00636F726E204D63427269646520496E6303
:10005B002E2020200D534D50544520496E7465724F
:10006B006661636520012056312E35370D00C2AF16
:10007B0075D00075816C43B0FF4390FF20B402C272
:10008B0095758921758804758DFD758BFDD28E75DF
:10009B0089237598D0787FE4F6D8FD751800751E06
:1000AB00149000007400F0A3A883B820F974FF909B
:1000BB00E800F0901523F090E000F0901522F07519
:1000CB00A015781E90E000E0F20890E800E0F2D274
:1000DB0094D29612019A902D8312024E902D961265
:1000EB00024E122D1A121C4E20B4031221D2121CD6
:1000FB002612217F90800274B5F0122D28122D1A32
:10010B001221D2122D1A122D1A122D1AC294122D3F
:10011B0028D294D22775B80075A811D2AF75129654
:10012B00901522E054FBF090E000F01214F312153E
:10013B006AC215C23FD201302A02C20175816C30EE
:10014B000144C28CC292758A00754C00C204D2461F
:10015B00D28CD2A9902D8312024E902D9612024E64
:10016B00120528302306120BF13001121202EB306C
:10017B0004EEC204B29412075B30010280E2C28C1F
:10018B00C2A9C246D2922022030216700218D8903E
:10019B00000075A0A07802E230E70BA3E583B4055D
:1001AB00F6C2380201EBD2387A301201EC7A3012F7
:1001BB0001EC7A381201EC7A801201EC7A0612010A
:1001CB00EC7A0C1201EC7A011201EC7A401201EC80
:1001DB007A5A12020B7A401201EC12022DB45AC158
:1001EB0022C0F030381775F00075A0A07802E2300D
:1001FB00E70700D5F0F30202087800EAF2D0F0220C
:10020B00C0F030381A75F00075A0A07802E230E724
:10021B000700D5F0F302022A75A0A07801EAF2D00C
:10022B00F022C0F030381975F00075A0A07802E20A
:10023B0030E70700D5F0F302024B75A0A07803E27C
:10024B00D0F022740093A312026CFA740093A32AC9
:10025B00FA1201EC740093A36006FA12020B80F4FD
:10026B002283227FBF93D37A851201ECE55175F07F
:10027B0000600475F00A842430FA12020BE5F024B6
:10028B0030FA12020B7A3A12020BE55275F000604B
:10029B000475F00A842430FA12020BE5F02430FACC
:1002AB0012020B7A3A12020BE55375F000600475DB
:1002BB00F00A842430FA12020BE5F02430FA120211
:1002CB000B7A2E12020BE55475F000600475F00AE0
:1002DB00842430FA12020BE5F02430FA12020B22BE
:1002EB00303A08E56930E00312030F303B08E5694B
:1002FB0030E103120446303C08E56930E203120496
:10030B0049C23A22E562C39561F4B412005003026C
:10031B000445A86275A01C74FEF2F5F075A01B7461
:10032B0001F20875A01CE56BF225F0F5F075A01B2A
:10033B00E4F20875A01C7428F225F0F5F075A01BEB
:10034B00E4F20875A01CE56AF225F0F5F075A01B28
:10035B00E4F20875A01CE551F225F0F5F075A01B31
:10036B00E4F20875A01CE5F0C313F275A01B740131
:10037B00F20875A01C74FEF2F5F075A01B7401F267
:10038B000875A01CE56BF225F0F5F075A01BE4F2E7
:10039B000875A01C7428F225F0F5F075A01BE4F28B
:1003AB000875A01CE56A2401F225F0F5F075A01B79
:1003BB00E4F20875A01CE552F225F0F5F075A01BD0
:1003CB00E4F20875A01CE5F0C313F275A01B7401D1
:1003DB00F20875A01C74FEF2F5F075A01B7401F207
:1003EB000875A01CE56BF225F0F5F075A01BE4F287
:1003FB000875A01C7428F225F0F5F075A01BE4F22B
:10040B000875A01CE56A2402F225F0F5F075A01B17
:10041B00E4F20875A01CE553F225F0F5F075A01B6E
:10042B00E4F20875A01CE5F0C313F275A01B740170
:10043B00F20888629060057406F022C23B22E562E6
:10044B00C39561F4B40C005003020527A86275A094
:10045B001C74FEF2F5F075A01B7401F20875A01C5C
:10046B00E56BF225F0F5F075A01BE4F20875A01C06
:10047B007428F225F0F5F075A01BE4F20875A01CAA
:10048B00E56A2404F225F0F5F075A01BE4F208757B
:10049B00A01C901563E0F225F0F5F075A01BE4F2BB
:1004AB000875A01CE5F0C313F275A01B7401F208CC
:1004BB0075A01C74FEF2F5F075A01B7401F20875A3
:1004CB00A01CE56BF225F0F5F075A01BE4F20875A6
:1004DB00A01C7428F225F0F5F075A01BE4F208754A
:1004EB00A01CE56A2405F225F0F5F075A01BE4F2DB
:1004FB000875A01C901564E0F225F0F5F075A01BB3
:10050B00E4F20875A01CE5F0C313F275A01B74018F
:10051B00F20888629060057406F0C23C22E55965CA
:10052B005A600812055B20232680F2302D05122815
:10053B0085800EE5636564600812068120231080B8
:10054B00F2E55F656060081206AC80F585605F229E
:10055B0075A01EA959E3FA75A01DE3FB0559C23915
:10056B00C229BB0006EA20280F803CEA30E7369010
:10057B00155CF0D228020680C228B4FE0DF51CF5DE
:10058B001D751800751E14020680B4800050057589
:10059B001D00805E751DFDD22490155DC0E0E4F05A
:1005AB00D0E002063DD229AD1DBDFE030205C9BD3B
:1005BB000003020619BDFD0302063D020680BB00C7
:1005CB0002801AF5F090155CE0251CC313B5F005FD
:1005DB00D2230206807455121645020680851EA092
:1005EB00A818F2251CF51C088818B80002051E0275
:1005FB00068090155CE075831C856282F074017532
:10060B00831BF00582E56165826024858262203957
:10061B001E75831C856282EAF0EB75831BF00582E5
:10062B00E561658260098582629060057406F0025F
:10063B00068030290990155DE0C313FAC229901585
:10064B005DE02AF0758318855E82EAF0302406C2DD
:10065B0024740180027400758317F00582E55D65D3
:10066B0082600F85825E90800274B5F09080057475
:10067B0006F00206802275A01AA963E3FA75A01989
:10068B00E3FB056375831F855C82EAF00582E55BFE
:10069B006582600385825C202002D299D2390205E3
:1006AB006B75A016A85FE2055FB4FE0BD230C231AA
:1006BB00C232C23302075A30300AB41302D231C2EB
:1006CB003002075A303110B42000505E901563F0A1
:1006DB00C231D23202075A30320A901564F0C2325C
:1006EB00D233806B30334BF87A11901563E02AFAD2
:1006FB00901564E02A547FC398702F901564E0F82E
:10070B00901563E09015652582F58274003583F5AD
:10071B0083E8F0D23C30E504D234800375671E9039
:10072B001522E054FDF090E000F0C231C232C2332A
:10073B00801DC231C232C23375831F855C82F005C6
:10074B0082E55B6582600385825C202002D2992260
:10075B0020930F203719D23774BF75F00A1215F892
:10076B00800D30370AC23774BF75F00B1215F87550
:10077B00A015791FE3FB90E800E0F36B5B60357B22
:10078B000833502EC0E090E000E030E61C75F0001E
:10079B0030E70375F01020E50343F04074B12BFAFA
:1007AB00EBF9121F2DD0E0800974B12BFA121FB593
:1007BB00D0E0DBCD75A015781EE2FA90E000E0F2F8
:1007CB006A5AFAEA541F605030E020D291C200C23C
:1007DB000110150DC23F30221C301F19121AAD80AB
:1007EB0037103F028032121AAD802D30E107202BDB
:1007FB0004D200C29130E304D201801C30221130AC
:10080B00E402D21530E211D201D2911220018008FC
:10081B0030E205D201122001227851E60846084643
:10082B00084660121208427002800B1208D1600653
:10083B007D16DDFE80F522900000E06026F97565DF
:10084B000030257D20267A7E107F008E828F83E0FC
:10085B00B4FF02806CF5F07851E6B5F002801040E1
:10086B0060D902805C74082EFEEF3400FF80DCA39D
:10087B00E0B4FF02804BF5F008E6B5F002800440CF
:10088B004080DEA3E0B4FF028037F5F008E6B5F058
:10089B00028004402C80CAA3E0B4FF028023F5F051
:1008AB0008E6B5F0028004401880B6E565B4000D8B
:1008BB00A3AB82AC83901520EBF0A3ECF005658025
:1008CB00A0C227E56522901520E0FBA3E0FCE565BF
:1008DB00B4000302091B8B828C83E0FEA3E0FFA311
:1008EB00E0F9700302090AA3E0B4FF0302091EB486
:1008FB008000500302094D0209A8D565028011EB57
:10090B002408FB901520F0A3EC3400FCF00208E166
:10091B00E56522E55CC3955BF489F0B5F000500307
:10092B0002091B8E828F83A85C75A01FE0F2A308BF
:10093B00D9FA885C202002D299D5650302091B02E3
:10094B00090AE562C39561F489F0B5F00050030222
:10095B00091B8E828F83A86275A01CE0D2E7F2750B
:10096B00A01B7401F2D903088022A308D902800FBF
:10097B00E075A01CF275A01B7400F2A308D9F1E07E
:10098B0075A01CF275A01B7401F2A308886290601D
:10099B00057406F0D5650302091B02090AE55EC35F
:1009AB00955DF489F0B5F000500302091B8E828F20
:1009BB0083A85EE075A018F275A0177401F2A30866
:1009CB00D90302090AE075A018F275A0177400F29A
:1009DB00A308D9F1885E90800274B5F090800574FD
:1009EB0006F0D5650302091B02090AE538C4540F4A
:1009FB00F5F0E53954F045F030E72530E622543F69
:100A0B00F5F0B43F028024900007E0B5F002801BA4
:100A1B00901500E0600AFAA3E0B5F002800DDAF75A
:100A2B0090153EE4F0A3F0A3F08008901536E5F0A6
:100A3B00F0D21622901536E0F5F0A3E53AC4540F28
:100A4B00F9E53B543049F025F0F5F0A3E53CC454EF
:100A5B000FF9E53D543049F025F0543FF5F0901572
:100A6B0036E5F0F022901536E0F5F0E53EC4540F74
:100A7B00F9E53F543049B5F002800B90153EE4F098
:100A8B00A3F0A3F08020C21E7903783E75A015E277
:100A9B00F5F0E0B5F0028002D21EF2121EAAD9EFD9
:100AAB00301E03021EB2227400B5520DB5530AB5A7
:100ABB0051077403B55400500122901526E060F9DC
:100ACB00FA7400F0A3A85E122178B4030040F87505
:100ADB00A018E0D2E7F2FB75A0177401F20875A01D
:100AEB00187408F22BFB75A0177400F20875A01888
:100AFB00EBF275A0177400F208885E75A08079027E
:100B0B0074B5F375A08079057406F3A3DAB9C21B2B
:100B1B0022900000E07005D226020B7575F0009054
:100B2B000005E0C395F0900003F075F00890000607
:100B3B00E095F0900004F0900000E0C226C3940210
:100B4B005002802604FA750513750400850406858A
:100B5B0005077907120BE7EAFB120B787907120BE3
:100B6B00E7DBF67905120BE7DAE2D22522C082C069
:100B7B0083A8058504A0850782850683E0F5F0E24E
:100B8B00C395F0C0D0120BBFE0F5F0E2D0D095F0DA
:100B9B00C0D0120BBFE0F5F0E2D0D095F0C0D01270
:100BAB000BBFE0F5F0E2D0D095F04003120BD3D0A1
:100BBB0083D08222C0E01582E582B4FF0215831830
:100BCB00B8FF0215A0D0E0227908E2F5F0E0F2E5DB
:100BDB00F0F0A308B8000205A0D9EF22E72408F72C
:100BEB0019E73400F722901400E0B44203020E39E7
:100BFB00543F2323900C0373020D0B00020F2D00A7
:100C0B00020FCE00020FDF00020FFC00020D0300EB
:100C1B0002100D000210330002106D000210FE00D6
:100C2B000212D5000212F90002131F000213390041
:100C3B0002134500021387000213E6000214BF00E3
:100C4B0002149B000214750002144C0002108F005A
:100C5B000210AF000212690002136B0002137A003C
:100C6B00020D0300020D0300020D0300020D030031
:100C7B00020D0300020D0300020D0300020D030021
:100C8B00020D0300020D0300020D0300020D030011
:100C9B00020D0300020D0300020D0300020D030001
:100CAB00020D0300020D0300020D0300020D0300F1
:100CBB00020D0300020D0300020D0300020D0300E1
:100CCB00020D0300020D0300020D0300020D0300D1
:100CDB00020D0300020D0300020D0300020D0300C1
:100CEB00020D0300020D0300020D0300020D0300B1
:100CFB00020D0300020D03007455121645C2232288
:100D0B00901401E0B4FE03020D2FB4FF03020D5D3E
:100D1B00B40003020D5DB4FD03020D5D7455121694
:100D2B0045C22322120D3A74AA121645C223227A07
:100D3B00079000007400F0A3DAFCD226D2257518B8
:100D4B0000751E14751F007400900005F07408A345
:100D5B00F022C21EF5F0202606900000E070030280
:100D6B000E28FBF51F7A01A9F0EA75F008A4240FF1
:100D7B00F582E5F03400F58389F0E0B5F0028003ED
:100D8B00020E1BD21EE582C39403F582E583940009
:100D9B00F583E0FCA3E0FDA3E0F9E51FC39A04C0D3
:100DAB00F075F008A4AFF0FEEA1475F008A4241057
:100DBB00F8E5F03400F5A0EA75F008A42410F582EC
:100DCB00E5F03400F583120E68ECF8EDF5A0E92C94
:100DDB00F58274003DF5837400C39582FE741495FF
:100DEB0083FF120E68900003E0C399F0A3E0940018
:100DFB00F0A3E0C399F0A3E09400F0120E77D0F0CB
:100E0B001B151FE51FB40003020D2FBB000C800D3B
:100E1B000ABB00028007DB028003020D72301E0644
:100E2B00E51F900000F074AA121645C22322A85C9D
:100E3B009000607900E993601AB40106744120B404
:100E4B00010475A01FF20908E8B55BE92020FAD26E
:100E5B009980F6885C202002D299C22322E0F212FC
:100E6B001EAADEF9BF00028002DFF222900014E519
:100E7B001F6029F8E0C39CAE82AF83A3E0950540C9
:100E8B000D8E828F83E0C399F0A3E09400F074077A
:100E9B002582F58274003583F583D8D82290000023
:100EAB00E0F5F0FA7B007E0D900003E02AFA740067
:100EBB003BFBA3DEF6900010AEF0BE0003020ED992
:100ECB007F08E02AFA74003BFBA3DFF6DEF290000A
:100EDB0003E0FFA3E0FE900800EE4F600FE02AFA5C
:100EEB0074003BFBA31FBFFFF01E80ED7E0F901520
:100EFB0000E02AFA74003BFBA3DEF67E0F90150F81
:100F0B00E02AFA74003BFBA3DEF67E20901546E048
:100F1B002AFA74003BFBA3DEF6900001EAF0A3EB88
:100F2B00F022900000E004B4FE087455121645023E
:100F3B000FCBF014F5F07408A42410F8E5F034008E
:100F4B00F5A07A04901401E0F2121EAADAF9E0B4CB
:100F5B00FE0E900000E014F07455121645020FCBF4
:100F6B00FDA3E0FCA3A982AA83900003E02CF0A3CD
:100F7B00E03400F0900005E0F5F0F2121EAAE0F26A
:100F8B00FB121EAAECF2121EAAEDF2121EAA74FF9D
:100F9B00F2121EAAF2121EAAF2121EAAF28A83895A
:100FAB0082A9F0E08BA0F3A309B900010BDCF4904C
:100FBB000005E9F0A3EBF0C226C22574AA12164570
:100FCB00C22322202606202503120B1C74AA1216FC
:100FDB0045C22322121E1F74AA121645C2232034A7
:100FEB000B901522E04402F090E000F0D297D296DD
:100FFB0022121C4E1221D212156A74AA121645C265
:10100B002322901401E0B4400040028013B40A0084
:10101B00400E900007F0121E1F74AA121645800591
:10102B007455121645C22322901401E0B40A0040F5
:10103B00028022FA780075A015F2121EAAE0B43FC6
:10104B00005012B43200400DF2DAEF74AA121645BA
:10105B00121E1F800A901500E4F07455121645C23B
:10106B002322780175A0149015467D20E2F0121E04
:10107B00AADDF9121E1F1221D212156A74AA1216BA
:10108B0045C2232290155CE0547FF56B901401E070
:10109B005407F569901402E0B41B004002741AF572
:1010AB006AC22322900009E075F01E700375F018D8
:1010BB00B4010375F019901401E0B418004001E479
:1010CB00901585F0901402E0B43C004001E49015BB
:1010DB0086F0901403E0B43C004001E4901587F0D7
:1010EB00901404E0B5F0004001E4901588F0D23D77
:1010FB00C22322901401E0700575F0188060B401D2
:10110B000575F0198058B4020575F01E8050B403B4
:10111B000575F01E8048B4040575F01E80407402FE
:10112B00900009F090150F7400F0A37400F0A374F5
:10113B0000F0A37400F0A37418F0A37400F0A37470
:10114B0000F0A37400F0A37400F0A37400F0A37478
:10115B0000F0A37400F0745512164502125A900059
:10116B0009F0901402E0B4180050B390150FF0F58D
:10117B0055901517F0901403E0B43C0050A0901557
:10118B0010F0F556901518F0901404E0B43C005094
:10119B008D901511F0F557901519F0901405E0B5D9
:1011AB00F0004003021129901512F0F55890151A12
:1011BB00F0C223901406E0B41804D2238005400338
:1011CB00021129901513F0F530901407E0B43C0090
:1011DB0040030211293023056003021129901514D5
:1011EB00F0F531901408E0B43C00400302112930B3
:1011FB0023056003021129901515F0F5329014099F
:10120B00E0B5F00040030211293023056003021101
:10121B0029901516F0F53390140AE0A2E09222A261
:10122B00E19205A2E2921FA2E3922AA2E4922BA2E0
:10123B00E5922DA2E6922EA2E79213900008F0D22F
:10124B0096202204C2018002D20174AA1216451202
:10125B001E1F1221D212156A12217FC22322900067
:10126B0009E075F01E700375F018B4010375F019E1
:10127B00901401E0B4180040028047901402E0B4CF
:10128B003C004002803C901403E0B43C00400280E0
:10129B0031901404E0B5F0004002802690151AF04E
:1012AB00901403E0901519F0901402E0901518F0CB
:1012BB00901401E0901517F074AA121645121E1F18
:1012CB0080057455121645C22322901401E0FBA32E
:1012DB00E0FA901522E04AF0FAA3E04BF090E80018
:1012EB00F090E000EAF074AA121645C22322901483
:1012FB0001E0F4FBA3E0F4FA901522E05AF0FAA314
:10130B00E05BF090E800F090E000EAF074AA1216AF
:10131B0045C2232290E800E0FB90E000E0FA74AABB
:10132B00121645EB121645EA121645C22322D201BC
:10133B00D29174AA121645C22322D291C200C201C5
:10134B0010150DC23F302210301F0D121AAD800840
:10135B00103F028003121AAD74AA121645C2232243
:10136B00202B04D200C29174AA121645C22322303C
:10137B002202D21574AA121645C22322901401E040
:10138B00A2E0921D900008E092E3C21D5002D21D14
:10139B00F075A015781B901402E0F9F208A3E0FA9F
:1013AB00F208A3E0F2FBC3740099748D9A74279B27
:1013BB0040030213DBC21D900008E054F7F09015B8
:1013CB001B7400F0A3F0A3F074551216450213E33F
:1013DB00121E1F74AA121645C22322900000E0FFB2
:1013EB00FA1216459000100FDF02804EE0121645E0
:1013FB002AFAA3E01216452AFAA3E01216452AFA96
:10140B00A3E01216452AFAA3E0FDA3E0FEA3E0FC3D
:10141B00A3E0A31216452AFAEC1216452AFAC0824B
:10142B00C0838D828E830CDC028009E01216452A64
:10143B00FAA380F3D083D08280AEEA121645C22382
:10144B00227F037E007A00903400E01216452AFAC0
:10145B00A3DEF7DFF59020007E10E01216452AFA86
:10146B00A3DEF7EA121645C223229015657F20E40E
:10147B00F0A3DFFC756700C234C235C2369015226B
:10148B00E04402F090E000F074AA121645C2232249
:10149B00E430350244013036024402FA121645900C
:1014AB0015657F20E01216452AFAA3DFF7EA12161C
:1014BB0045C22322901401E0541F75F010A42400A0
:1014CB00F582E5F03435F58375A0147801121C39DB
:1014DB00A85E122178B4100040F890140112151B6D
:1014EB0074AA121645C223227C20EC1475F010A4AA
:1014FB002400F582E5F03435F583E030E70FA85E84
:10150B00122178B41000500280F612151BDCDB227E
:10151B00E0D2E775A018F2FB75A0177401F20875FD
:10152B00A0187400F275A017F208A37A0DE075A04D
:10153B0018F22BFB75A0177400F208A3DAEF75A055
:10154B0018EBC313F275A0177400F208885E75A030
:10155B0080790274B5F375A08079057406F32212B5
:10156B002178B4080040F874BF855E82758318F04B
:10157B00FB7583177401F074030582758318F02BC8
:10158B00FB758317E4F00582758318F0758317F0EC
:10159B000582758318F0758317F0C082900009E0FF
:1015AB00D0820582758318F02BFB758317E4F0E569
:1015BB00350582758318F02BFB758317E4F0E53442
:1015CB000582758318F02BFB758317E4F005827584
:1015DB008318EBC313F0758317E4F0058285825EE5
:1015EB0090800274B5F09080057406F022FBE55EE6
:1015FB00C3955DF4B4030050030215F9EBA85E75B7
:10160B00A018F275A0177401F20875A018E5F0F296
:10161B002BFB75A0177400F20875A018EBC313F21F
:10162B0075A0177400F208885E75A080790274B5F6
:10163B00F375A08079057406F322C0E0C082C083E5
:10164B0075831F855C82F0E55C04F583B55B072031
:10165B0020FAD29980F685835C202002D299D08320
:10166B00D082D0E02275A891C28CC28EC28F902DF1
:10167B00A912024E902DB912024E902DE112024E7C
:10168B00C20BC20DC212C20FC20CC210C20EC207D5
:10169B00851211758A00754C00752940752A0175E4
:1016AB005500755600755700755800753300901529
:1016BB001BE0F530A3E0F531A3E0F532C2AF75B80E
:1016CB000675A81FD246D28CD2AFC223121C26128B
:1016DB00052830230D75A891C28CC28E120BF10216
:1016EB0018BE100C183004E7C2041202EB12075B91
:1016FB003001DC75A891C28CC28E0218BEE539543C
:10170B000375F00AA4F8E538540F28200E09B41518
:10171B00BED20E7A0080B8F890172BEA54032373CD
:10172B008006800A800E8028B8165E0A80A1B81742
:10173B00580A809BB818030A8095B8004C75461858
:10174B0075127875295BC206902E2412024E803ECC
:10175B00B8192075461E751296752915C206902E5E
:10176B003612024EE53930E208D206902E3F1202B5
:10177B004E801BB8001375461975127D75294DC225
:10178B0006902E2D12024E8005C20E0216DA902DF7
:10179B00C712024EC2AF854341854442D2AFE541E9
:1017AB0075F014A4F541A8F0E54275F014A428F5E2
:1017BB0042754E00754D00D210D20FE539540375AA
:1017CB00F00AA4F5F0E538540F25F004F548F5546C
:1017DB00E53B540775F00AA4F5F0E53A540F25F0F4
:1017EB00F549F553E53D540775F00AA4F5F0E53CD2
:1017FB00540F25F0F54AF552E53F540375F00AA452
:10180B00F5F0E53E540F25F0F54BF551D23A121C8D
:10181B0026C202C218C219740AF56630B402C2900D
:10182B001205283023030216E020100C75A891C274
:10183B008CC28E752800807B30190FC21930030AB9
:10184B00D56607740AF566121B63301836C2181278
:10185B00075B30010975A891C28CC28E8055300D83
:10186B000B1209F6902DC712024E8017902DD41231
:10187B00024ED296E511600BD51108D236C201C2C9
:10188B0022803030021DC202301603120A3F301B79
:10189B0003120AB212082430130312228E1202EB27
:1018AB0012027230170AC217301605C216120A70CE
:1018BB0002182B121C2630B402D290D297D29690DB
:1018CB001522E04409F090E000F002014775A89161
:1018DB00C28CC28EC215C23FC21AC218901522E02A
:1018EB0054FEF090E000F0902DB112024E121AADA2
:1018FB0020426420413A20402575461875400090DF
:10190B001554E0B4E90C902E2412024E901554029B
:10191B001975902E1B12024E901554021975902EAC
:10192B002D12024E90155675461975400002197509
:10193B00304012902E3612024E90155A75461E7577
:10194B004000021975902E3F12024E9015587546A5
:10195B001E754004021975902E4812024E901558B0
:10196B0075461E754000C240C241E0A3750F00F5DD
:10197B000EE0F50D754700750936750C00750B0AF1
:10198B00750A01D209850E4F121C26C2AF75B8021B
:10199B00850E8A202E0D902DF412024E75A81BD2A7
:1019AB008C802D75A81FC28B902DB912024E902ED4
:1019BB000E12024E204113902E1B12024E74EA752A
:1019CB000F00F50E74C2F50D8006902E4812024ED4
:1019DB00C246C28DC28FD2AFC223740AF56630B431
:1019EB0002C290120528302306120BF1200133306E
:1019FB000211C20212082430130312228E1202EBC0
:101A0B001202723018DDC21812075B200114301558
:101A1B000FC29230B402D290902E0112024E800E61
:101A2B0080C175A891C28CC28E752800805F12058B
:101A3B0028202332300228C2021202EB12075B204D
:101A4B00013B20151AD29230B402C290202E08907E
:101A5B002DF412024E808C902E0E12024E8084308A
:101A6B0018CCC21880C8D29175A891C28CC28EC2F4
:101A7B0015C23FD201752800120BF18010D291755F
:101A8B00A891C28CC28EC215C23F75280030B40219
:101A9B00D290901522E04401F090E000F0D2960233
:101AAB000147121C2690150FE0F555A3E0F556A340
:101ABB00E0F557A3E0F558A3E0F530A3E0F531A32B
:101ACB00E0F532A3E0F533A3E0F54BA3E0F54AA331
:101ADB00E0F549A3E0F548303D14901585E0F54B52
:101AEB00A3E0F54AA3E0F549A3E0F548C23D900019
:101AFB0009E070087528007568048027B401087523
:101B0B002801756804801CB40308752804756801E6
:101B1B008011B404087528027568018006752803C6
:101B2B007568017536FC7537BFE54875F00A848515
:101B3B00F0384540F539E54975F00A8485F03AF5FA
:101B4B003BE54A75F00A8485F03CF53DE54B75F0B5
:101B5B000A8485F03EF53F2290400374C2C2AFF079
:101B6B00904000E0E0F4FCE0F4FD9040037436F0AC
:101B7B00904000E4F0F0D2AF202C43ED13547FFDE6
:101B8B00EC132403FCED3400FDC3E5349CFC9060A6
:101B9B0003F0E5359DFD906003F075F00030E70331
:101BAB0075F0FFAEF0C390155EE03CFCF0A3E03D9A
:101BBB00FDF0A3E03EFEF020E70C4D4C702EC22C46
:101BCB00AD2CAC2D804775F00AF47013EDF4700F4B
:101BDB00ECF4B45000500803030303540FF5F0E585
:101BEB002CC395F0FDE52D9400FC802175F00AEED9
:101BFB007011ED700EECB450005008030303035446
:101C0B000FF5F0E52C25F0FDE52D3400FC75A0401B
:101C1B007801EDC2AFF2ECF2D2AF22D22CE49015E8
:101C2B005EF0A3F0A3F0AD2CAC2D121C18227A1091
:101C3B008003121EAAE2F0DAF9FAE0C39A70FB12E3
:101C4B001EAA22120D3A121DD6903440E0B4550D47
:101C5B00902000E0FCB4FE004006021CFB021D4E6F
:101C6B00902003E0A3F8C3740098E0F8740C98502C
:101C7B0003021CFB90200075A0007800ECF27D00A5
:101C8B00FE121EAAE0FBF2121EAAE0FAF2121EAA24
:101C9B007F0DE0F22CFC74003DFD121EAADFF3BE9B
:101CAB000004D226804AC226902010781075A0001E
:101CBB007F08E0F22CFC74003DFD121EAADFF3DE60
:101CCB00EF7E08E0F2121EAADEF9900003E0FFA3FC
:101CDB00E0FE90280075A0087800EE4F6012E0F24D
:101CEB00121EAA2CFC74003DFD1FBFFFED1E80EAE7
:101CFB007F0F780075A015903400E0F2121EAA2C0D
:101D0B00FC74003DFDDFF37F0F780F75A015903449
:101D1B0010E0F2121EAA2CFC74003DFDDFF37F20B5
:101D2B00784675A015903420E0F2121EAA2CFC7494
:101D3B00003DFDDFF3ED8AF0B5F008EC8BF0B5F06C
:101D4B00028030901522E054FDF090E000F0D23587
:101D5B00C297C296122D1A122D1AD297D2967C20A8
:101D6B009034FF7A107400A3F0DAFCE0B400FCDCD2
:101D7B00F28010900000E06006C226D2258004D2CB
:101D8B0026C2257D04785590150FE0F6A308DDFAE1
:101D9B007D047830901513E0F6A308DDFA90000867
:101DAB00E0A2E09222A2E19205A2E2921FA2E392AC
:101DBB002AA2E4922BA2E5922DA2E6922EA2E79202
:101DCB0013202204C2018002D20122902D4375A060
:101DDB000078007A10E493F2121EAADAF8902D53D1
:101DEB0075A01578007A0FE493F2121EAADAF89018
:101DFB002D7475A015780F7A0FE493F2121EAADAE0
:101E0B00F8902D5E75A01578467A16E493F2121EA3
:101E1B00AADAF822202606202503120B1C120EA884
:101E2B00780075A000902000E2FC121C39EC7003C6
:101E3B00021E73C31304FC121C39DCFB900003E07D
:101E4B00FCFFA3E0FD7A04EDC313FDEC13FCDAF702
:101E5B00EF540F60010CBC0002800D780075A008D8
:101E6B00902800121C39DCFB780075A0159034000B
:101E7B00121C39780F75A015903410121C39784646
:101E8B0075A015903420121C39785675A015903416
:101E9B0030121C399034407455F0E0B455FC22A339
:101EAB0008B8000205A022901537E0540F232390A9
:101EBB001EBE73021EFF00021F1900022005000246
:101ECB00205A0002207F0002208B00022097000284
:101EDB0020A30002210E0002212800022142000251
:101EEB00215D00021EFE00021EFE00021EFE00020D
:101EFB001EFE0022901537E05430FA334A5450FA44
:101F0B00A3E0543F901524F0901525EAF02290158C
:101F1B0038E0543FD2E7FA901524E0F9901525E00C
:101F2B00F5F0301D048A588933122178B40500402E
:101F3B00F8758318855E82EAF07583177401F005D6
:101F4B00827583187401F02AFA7583177400F005F3
:101F5B0082758318E5F0644003542045F020220776
:101F6B00200D09440880053001024408F02AFA7557
:101F7B0083177400F00582758318E9543FF02AFA31
:101F8B007583177400F00582758318EA03547FF08C
:101F9B007583177401F0058285825E90800274B59B
:101FAB00F09080057406F0C22122122178B4030050
:101FBB00500280F6758318855E82EAF0758317747C
:101FCB0001F005827583187408F02AFA758317746B
:101FDB0000F00582758318EA03547FF0758317743C
:101FEB0001F0058285825E90800274B5F0908005C9
:101FFB007406F0C22122743F8006C221901538E08E
:10200B00543FD2E7FA122178B40300500280F675E0
:10201B008318855E82EAF07583177401F00582756B
:10202B0083187408F02AFA7583177400F00582750B
:10203B008318EA03547FF07583177401F0058285CA
:10204B00825E90800274B5F09080057406F0229049
:10205B001538E0543FFA901526E0B40A02801204BA
:10206B00F0F9E58229F58274003583F583EAF0D225
:10207B001BC22122901538E0543FFA79180220AF89
:10208B00901538E0543FFA79190220AF901538E0DB
:10209B00543FFA791A0220AF901538E0543FFA7981
:1020AB001B0220AFE562C39561F4B40500500280BA
:1020BB00F375831C75A01B85628274FF4480FBF053
:1020CB007401A882F205827400F02BFB7400A882C5
:1020DB00F20582E9547FF02BFB7400A882F2058293
:1020EB00EAF02BFB7400A882F20582EB03547FF01D
:1020FB007401A882F205828582629060057406F0F5
:10210B00C22122901537E0232354C0F9A3E0543F9A
:10211B0049F9901522E049F090E000F02290153734
:10212B00E0232354C0F9A3E0543F49F9901523E071
:10213B0049F090E800F022901537E0232354C0F9C2
:10214B00A3E0543F49F4F9901522E059F090E000D8
:10215B00F022901537E0232354C0F9A3E0543F49F4
:10216B00F4F9901523E059F090E800F022E55EC3F6
:10217B00955DF4229060027415F0906000202D04A0
:10218B00741B80027413F07407F0A3202D0474BB2E
:10219B00800274CCF09060047408F09060027405B7
:1021AB00F09060057406F09080027415F09080003A
:1021BB00741BF07407F0A374CCF09080047408F0D7
:1021CB009080057404F022121C26C203901546E081
:1021DB00F52B6002D203A3A3A3E0F52DA3E0C0E08F
:1021EB0054FEC39432F52CE52D9400F52D30B4023A
:1021FB00D2959040037476F09040017F32E52C2409
:10220B0002F52CF0E52D3400F52DF0122D3ADFED13
:10221B007F19E52CC39402F52CF0E52D9400F52DD8
:10222B00F0122D3ADFECD0E0F52CF0E52DF020B4D8
:10223B002774E775F0007F08122CE1903421E0F54C
:10224B00F0A3E07F10122CE1A3E0F5F0A3E07F0FE9
:10225B00122CE1D297A3F52D12226722900009E0F0
:10226B00B4000590154C8013B4010590154E800BEE
:10227B00B402059015528003901550E0F535A3E09C
:10228B00F53422C0D0C0E0C0F0C082C083E55EC38D
:10229B00955DF4B40700500302232D758318855EFA
:1022AB008274BFF0F5F07583177401F005827583A6
:1022BB0018740DF025F0F5F0758317E4F0058275B1
:1022CB008318E54BF025F0F5F0758317E4F00582E4
:1022DB00758318E54AF025F0F5F0758317E4F005E2
:1022EB0082758318E549F025F0F5F0758317E4F056
:1022FB000582758318E548F025F0F5F0758317E432
:10230B00F00582758318E5F003547FF0758317E4AD
:10231B00F0058285825E90800274B5F09080057422
:10232B0006F0D083D082D0F0D0E0D0D0222046036C
:10233B00D28C32C0D0C0E0D214300D02B2967402EF
:10234B00C28CC58AD28CF54FE4C54C308D07047016
:10235B00027403C28DF550C3E54F948AE550940087
:10236B00401BC3E529954FE52A95504004D20880C0
:10237B001374B5954F74029550C2085007C20BC227
:10238B000D02245930080D30070A200A28C2070510
:10239B0047022459200B71A208E53713F537E536B0
:1023AB0013F536B4FC7EE537B4BF79300807D20A93
:1023BB00D20702245920B5FD30B5FDC294D2177453
:1023CB0000B54808B54905B54A028016E53F5407E4
:1023DB0075F00AA4F5F0E53E540F25F0F54BF551D9
:1023EB00D23A750938750B08750A08754700D20B78
:1023FB00C20AC207300F57754500754E00754D0068
:10240B00D28ED28FC20F8046C000A208A809E61355
:10241B00F6D000D50A0E0509750A08D50B06C20BB6
:10242B00D20DD20C300804D20780230547C207E532
:10243B004354F02544C4F50FE54F54F02550C42503
:10244B004350020544C3950FF54350021544D0E0A9
:10245B00D0D032204603022474C0E0054CE54C700A
:10246B0005D204754C03D0E032C0D0C0E0C0F0C040
:10247B0082C083300911301507300504D2968002D3
:10248B00B296C207022526C000A809E630E00E303E
:10249B001507300504D2968002B296D20703F6D008
:1024AB00000547E50AC333F50A5070750A010509A3
:1024BB00D50B68750936750B0A7547008548548529
:1024CB004953854A52854B51D23AE54875F00A84F7
:1024DB0085F0384540F539E54975F00A8485F03AC1
:1024EB00F53BE54A75F00A8485F03CF53DE54B7507
:1024FB00F00A8485F03EF53FD28F302E1ED5681B37
:10250B00B209750C00C28C758AFE756801E52854FA
:10251B0007B40200502F756804802AB209850E4F4C
:10252B00E50CC3950D4002054F050CC28CE4C39519
:10253B004F258AF58AD28C201A0BE509B43B06D2BB
:10254B001AD218D294D083D082D0F0D0E0D0D0322F
:10255B002046030227C7C0D0C0E0E54E6004154EED
:10256B008019E54D601AC3E4954D754D00C28E255B
:10257B008C5004D28E8009F58CD28ED0E0D0D03224
:10258B00C21AE545700D200D1320B5FD30B5FDC207
:10259B00948009B40206D21AD294D218C0F0C08328
:1025AB00C082200D030226E8201A0C101406C20D5F
:1025BB00C20BD20F0226E853A8FB854C17858A164F
:1025CB00E547A20785441485431543A8049211F5EA
:1025DB00F0B428004003022666C3742895F023F557
:1025EB00139415400BC20DC212C20BD20F0226E878
:1025FB00E514C313C51513F51420110BC39516E57C
:10260B00159517400280021513E5148513F0A4F5F8
:10261B001685F017E5158513F0A42517C313C516FA
:10262B0013C516C313F517E51613F516E517C313E4
:10263B00F515E51613C515C313C51513F51425416B
:10264B00F541E5153542F542E5162541F54DE51702
:10265B003542F54E154ED2120226F0942823F5136F
:10266B009415400BC20DC212C20BD20F0226E8E525
:10267B0014C313C51513F51420110BC39516E515CB
:10268B009517400280020513E5148513F0A4F51687
:10269B0085F017E5158513F0A42517C313C516137D
:1026AB00C516C313F517E51613F516E517C313F582
:1026BB0015E51613C515C313C51513F514C3E5415D
:1026CB009514F541E5429515F542C3E5419516F58F
:1026DB004DE5429517F54E154ED212800885424EA8
:1026EB0085414D154EE545B403028008B40102D275
:1026FB00190227B7300D5A301257C297901522E0A6
:10270B0054F6F090E000F0851211E539540375F0A2
:10271B000AA4F5F0E538540F25F0F548E53B5407CE
:10272B0075F00AA4F5F0E53A540F25F0F549E53DAF
:10273B00540775F00AA4F5F0E53C540F25F0F54A63
:10274B007400B5481CB54919B54A160548054B80A8
:10275B004BD297901522E04408F090E000F0121C49
:10276B00260548E548B546347548000549E549B4A2
:10277B003C2A754900054A300610E54A75F00A8473
:10278B00E5F0600674022548F548E54AB43C0D7542
:10279B004A00054BE54BB41803754B00854854852F
:1027AB004953854A52854B51D202D23A054553457E
:1027BB0003D082D083D0F0D0E0D0D032C0D0C0E0F4
:1027CB00C0F0C083C082301503022863103D3D0565
:1027DB0048E548B546487548000549E549B43C3ECF
:1027EB00754900054A30411020400DE54A75F00A45
:1027FB0084C5F06003754802E54AB43C21754A0074
:10280B00054BE54BB41817754B008012901585E0FE
:10281B00F54BA3E0F54AA3E0F549A3E0F548E54BFA
:10282B00B53035E54AB53130E549B5322BE548B51C
:10283B003326D291302B0D200506D215D23F8018AE
:10284B00D20180143000052005F680EE85554B85AE
:10285B00564A855749855848D202C21A20B5FD30D1
:10286B00B5FDC294901522E04401F090E000F0D049
:10287B0082D083D0F0D0E0D0D032E564C3956385AD
:10288B00631BB407005003022B76122B77B4F06650
:10289B00122B7720E75EB47F5D122B7720E755B4C0
:1028AB007F02800B2409F5F0900007E0B5F047128A
:1028BB002B7720E73FB4023E122B7720E736B4107C
:1028CB00028008B430028003B47F2B122B7720E7F1
:1028DB0023F51AB401028021B40202801CB4030256
:1028EB008017B41503022980B41603022980B4178C
:1028FB0005022980151B022B70E564C39563B40F89
:10290B00005003022B76122B7720E7E8C394307527
:10291B00F00AA4F51C122B7720E7D9C39430251CA1
:10292B00F51C122B7720E7CCB400CB122B7720E7CA
:10293B00C3C39430F51D122B7720E7B8B400B71240
:10294B002B7720E7AFC3943075F00AA4F51E122B3A
:10295B007720E7A0C39430251E75F00AA4F51E85D9
:10296B00F01F122B7720E78CC39430251EF51EE544
:10297B001F3400F51F122B7730E73BB4F73BE51AFA
:10298B00B40104C201804BB403028046B4020302BB
:10299B002A95B41527D291C200C20110150DC23F62
:1029AB00302210301F0D121AAD8008103F02800329
:1029BB00121AAD022AE6022B700228FFB416083059
:1029CB0022F1D215022AE6B41705D201022AE60239
:1029DB002B70122178B40500500280F67583188590
:1029EB005E82E51C4480F519B481004000F07583CC
:1029FB00177401F00582758318E51DC3C23E94035D
:102A0B00400EF51D94034004F51DD23E740D80025B
:102A1B007401F02519F5197583177400F00582758B
:102A2B008318E51E33E51F3330E20244105413C5FF
:102A3B001D600920E104744080027420451DF51DC2
:102A4B00E51AB403067408451DF51DE51D103E027D
:102A5B004408F02519F5197583177400F005827574
:102A6B008318E51E547FF02519F51975831774002B
:102A7B00F00582758318E51903547FF0758317747D
:102A8B0001F0058285825E022ADA122178B40300F6
:102A9B00500280F6758318855E82E51C4480F5191B
:102AAB00F07583177401F005827583187408F0258F
:102ABB0019F5197583177400F00582758318E519DC
:102ACB0003547FF07583177401F0058285825E9045
:102ADB00800274B5F09080057406F074F075831C59
:102AEB00856282F0740075831BF00582E561658257
:102AFB006073858262747F75831C856282F07400BB
:102B0B0075831BF00582E56165826059858262746D
:102B1B000375831C856282F0740075831BF005823C
:102B2B00E5616582603F858262740275831C8562F4
:102B3B0082F0740075831BF00582E5616582602568
:102B4B0085826274F775831C856282F074007583CD
:102B5B001BF00582E5616582600B858262906005E2
:102B6B007406F08000851B630228852275831A8505
:102B7B001B82E0051B22C0D0C0E0C082C08310992D
:102B8B000C109826D083D082D0E0D0D032C299E5F9
:102B9B005B655C7005C220022BB2D220855B82057F
:102BAB005B75831FE0F599022B89E59975831E856B
:102BBB005A82F075831D209A04740080027401F010
:102BCB00A3E5596582600385825A022B89C0D0C068
:102BDB00E0C082C083908005E030E103022C7E9040
:102BEB008005E030E203022CC9906005E030E10380
:102BFB00022C13906005E030E205022C5280D6D0F7
:102C0B0083D082D0E0D0D032E561656270099060EC
:102C1B00057404F0022BFE202D1D9060027415F03C
:102C2B0075831B856182E06008906000741FF080E3
:102C3B0006906000741BF075831C856182E09060C8
:102C4B0003F00561022BFE906001E075831985642A
:102C5B008220E504740080027401F0906003E0753B
:102C6B00831A856482F0A3E56365826003858264C1
:102C7B00022C08E55D655E700F9080057404F09082
:102C8B00800274A5F0022BEA9080027415F0758314
:102C9B0017855D82E06008908000741FF0800690BD
:102CAB008000741BF0758318855D82E0908003F0C3
:102CBB00055DB48100400400000000022BEA908007
:102CCB0003E0758316856082F0A3E55F6582600380
:102CDB00858260022BF4D295C295C0E07410C39F1D
:102CEB00FE600CD0E033C5F033C5F0DEF8C0E0D0A9
:102CFB00E0C29020F704C2978002D297D295C2957A
:102D0B0033C5F033C5F0DFEBD290D295C295227A62
:102D1B003EEAC0E0122D28D0E0FADAF5227A007BE9
:102D2B0020DAFEDBFC227A007B0ADAFEDBFC227A5D
:102D3B00007B32DAFEDBFC22000000000000080AF8
:102D4B000202000000000000000000000000000074
:102D5B0000000000000100040047C744E8397B393C
:102D6B006CEE00E5CDBECEBD0000000000180000EB
:102D7B000000000000008D27010144696769746140
:102D8B006C2042696E6C6F6F702000020156657289
:102D9B0073696F6E20312E35372020202000010102
:102DAB00526561642000010147656E202000010619
:102DBB002D2D3A2D2D3A2D2D2E2D2D0002014C6F40
:102DCB00636B65642020202000020153656C662034
:102DDB0047656E20200002014177616974696E6757
:102DEB0020534D505445202000020152756E6E69E0
:102DFB006E6720202000020149646C696E672020F9
:102E0B002020000201562D53796E632020202000D4
:102E1B00020B32332E39373600020B3234206670F8
:102E2B007300020B32352066707300020B333020B7
:102E3B0066707300020B32392E39376400020B3285
:062E4B00392E39376E003C
:00000001FF
